:020000040000FA
:06000000020091022C2217
:03002300022900AF
:03002B00022C366E
:10003B00022B1B53D9BF79012200000080FB120059
:10004B003EB9000302008BE4901000784F790A80D0
:10005B0002F0A3D8FCD9FA90194EAA82AB83900078
:10006B00A078F679018015E493A3AC82AD838A82E4
:10007B008B83F0A3AA82AB838C828D83D8E9D9E7DB
:10008B00122CB812004475D0007581BF7510007525
:10009B001110020049506C656173652070726573B5
:1000AB007320616E79206B657920746F20636F6E9E
:1000BB0074696E75652E2E2E203F007C205452499C
:1000CB0047207C203530306E732F64207C203235F6
:1000DB002E30562F64207C2032352E30562F642044
:1000EB007C3F007C2053796E63207C20496E74200A
:1000FB007C205A20434841207C205A2043484220F0
:10010B007C20464654207C3F0032352E30562F64DF
:10011B003F00496E743F0053796E633F00000259F4
:10012B00802054524947203F000000203530306E6C
:10013B00732F64203F2032352E30562F64203F2002
:10014B0032352E30562F64203F2053796E63203F7B
:10015B0000000020496E74203F00000000205A2050
:10016B00434841203F0000205A20434842203F0093
:10017B000020464654203F00000000000000000015
:10018B0000000000000101400707CAC0E0E6F0A331
:10019B0008DAFAD0E0FA22C3E498F8E499F91201EC
:1001AB00E38026C3E49AFAE49BFBE920E7E912011A
:1001BB00E3E498F8E499F922C3E498F8E499F91286
:1001CB0001E3E498F8E499F9C3E49AFAE49BFB227F
:1001DB00EB20E7CFE920E7E0B90010BB0008E88A85
:1001EB00F084F8AAF022E4FBC8FA22EB70227B1011
:1001FB00C833C8C933C9335007C39AC3DBF280066F
:10020B009A50012ADBEAC833F4C8C933F4C9FA227D
:10021B0075F008E4C833C8C933C933C99AC99B50B0
:10022B0004C92AC93BD5F0ECFBC833F4C8E4C9FABE
:10023B0022600D08C6A2E713C618C613C6D5E0F395
:10024B0022700422600D18C6C333C608C633C6D548
:10025B00E0F41822251010AF08F51040021511809C
:10026B0008F51040021511D2AF22C0D0251010AFE7
:10027B0008F510500205118008F51050020511D237
:10028B00AFD0D0222510F58210AF08F51040021523
:10029B00118008F51040021511D2AF85118322256C
:1002AB0010F582E43511F583222510C582C0E0E5F7
:1002BB001134FFC583C0E0E510C3958224F9F8E43F
:1002CB00C5A8858311858210C5A8E8CEF0A3E520CB
:1002DB00F0A37808E608F0A3DEFAEFF0A3E581249B
:1002EB00FBF8E608F0A3E608F0A30808E608F0A37D
:1002FB00E608F0A315811581D0E0FED0E0F815815A
:10030B001581E8C0E0EEC0E022851183851082E004
:10031B00A3FEE0A3F5207808E0A3F608DFFAE0A33C
:10032B00FFE0A3C0E0E0A3C0E0E0A3C0E0E0A3C017
:10033B00E0E4C5A8858210858311C5A8D083D0823F
:10034B002274028000C0E0F40412028FD0E012018C
:10035B009522D083D082C5F0E493A3C5F0C395F06A
:10036B00F5F0E493A3C395F04005E5F0048001E4B8
:10037B0075F002A42582F582E5F03583F583E493CD
:10038B00A3C0E0E493C0E022D083D082E9C0E0E4D4
:10039B0093A3C386F0C5F095F0F908E493A386F018
:1003AB00C5F095F0700BE493A3C3994005E9048065
:1003BB0002A3E475F002A42582F582E5F03583F5FE
:1003CB0083D0E0F9E493A3C0E0E493C0E022D083B0
:1003DB00D082CCC0E0E493A360061204031470FA3D
:1003EB00E493A360061204221470FAD0E0FCE493A9
:1003FB00A3C0E0E493C0E022C0E0E493A3D39C50FD
:10040B0010E493A3C39C400AD0E0D0E0D0E00203F9
:10041B00F6A3A3A3D0E022C0E0E493A36C7009D0B1
:10042B00E0D0E0D0E00203F6A3A3D0E022008040AE
:10043B00C020A060E0109050D030B070F008884819
:10044B00C828A868E8189858D838B878F8048444AD
:10045B00C424A464E4149454D434B474F40C8C4CB9
:10046B00CC2CAC6CEC1C9C5CDC3CBC7CFC0282425F
:10047B00C222A262E2129252D232B272F20A8A4AB9
:10048B00CA2AAA6AEA1A9A5ADA3ABA7AFA0686464D
:10049B00C626A666E6169656D636B676F60E8E4E59
:1004AB00CE2EAE6EEE1E9E5EDE3EBE7EFE01814108
:1004BB00C121A161E1119151D131B171F109894989
:1004CB00C929A969E9199959D939B979F90585451D
:1004DB00C525A565E5159555D535B575F50D8D4D29
:1004EB00CD2DAD6DED1D9D5DDD3DBD7DFD038343CF
:1004FB00C323A363E3139353D333B373F30B8B4B29
:10050B00CB2BAB6BEB1B9B5BDB3BBB7BFB078747BC
:10051B00C727A767E7179757D737B777F70F8F4FC8
:10052B00CF2FAF6FEF1F9F5FDF3FBF7FFF004020DD
:10053B0060105030700848286818583878044424E4
:10054B0064145434740C4C2C6C1C5C3C7C024222A6
:10055B0062125232720A4A2A6A1A5A3A7A064626A4
:10056B0066165636760E4E2E6E1E5E3E7E0141216F
:10057B006111513171094929691959397905452594
:10058B0065155535750D4D2D6D1D5D3D7D03432356
:10059B0063135333730B4B2B6B1B5B3B7B07472754
:1005AB0067175737770F4F2F6F1F5F3F7F00402025
:1005BB006010503070084828681858387804442464
:1005CB0064145434740C4C2C6C1C5C3C7C02422226
:1005DB0062125232720A4A2A6A1A5A3A7A06462624
:1005EB0066165636760E4E2E6E1E5E3E7E014121EF
:1005FB006111513171094929691959397905452514
:10060B0065155535750D4D2D6D1D5D3D7D034323D5
:10061B0063135333730B4B2B6B1B5B3B7B074727D3
:10062B0067175737770F4F2F6F1F5F3F7F00000004
:10063B0000000000000000000000000000000000AF
:10064B00600000000000000070000000003000009F
:10065B007C000000003F80007E000000003FF8009F
:10066B007F8000000001F8007FE00000000108001F
:10067B003FF80000000100000FFE00000001000029
:10068B0003FF80000021000000FFF000003F00008E
:10069B00001FFC00183FF8000007FF801807F80048
:1006AB000000FFE01800180000003FFC18000000DD
:1006BB00000007FF9C007800000000FFFC3FF800E3
:1006CB000000003FFC3FF8000000001FFC1800007A
:1006DB00000001FFFC06000000000FFFFC01800082
:1006EB000000FFFFFC00E0000007FFFFFC07F80025
:1006FB00007FFFFFE03FF80003FFFFFE003F00001D
:10070B001FFFFFF0000C00007FFFFF000003000045
:10071B007FFFF0000000C0007FFF8000000038006A
:10072B007FFC0000000008003FFC000000300000D0
:10073B000FFF80000030200001FFE0000010700070
:10074B00003FFC00000020000007FF8000000000BD
:10075B000001FFF00000000000003FFC0000000063
:10076B0000000FFF80000000000001FFE000000010
:10077B007000007FF80000007C00001FF8300000C4
:10078B007F000007FC3F80007FE00001FC0F800032
:10079B003FFC00007C0100003FFF00003C0180009B
:1007AB003FFFE0001C0180003FFFF8000008000045
:1007BB0038FFFF00183F0000383FFFE0183F800074
:1007CB003807FFFC182280003801FFFF98228000B9
:1007DB0038003FFFF813800078003FFFFC03000058
:1007EB00780039FFFC0000007800383FFC018000E6
:1007FB0078003807FC3F800078003801FC3F800010
:10080B00780038003C3000007C0038001C0C0000E5
:10081B007E0038001C0600003F0038001C018000E1
:10082B001FC038001C0080000FE038001C000000C7
:10083B0003E018001C00000000E000001C0000009A
:10084B00000000001C0000000000000E1C00000057
:10085B006000000FFC3C00007C00000FFC3C7000B3
:10086B007F000007FC3C78007FE00001FC21780052
:10087B007FF800007C2108007FFF00000C2108009E
:10088B003FFFE000003F080007FFF800183FF800AB
:10089B0001FFFF00181EF800003FFFE01800780072
:1008AB000007FFFC1C0000000001FFFF9C30000054
:1008BB0000003FFFFC300000000007FFFC30000091
:1008CB00000001FFFC0000007000003FFC00000076
:1008DB007C000007FC0400007F000001FC06000008
:1008EB007FE000003C0500007FF800000004800062
:1008FB003FFF0000000460003FFFE000003E3000BF
:10090B003FFFF800183FF80038FFFF001807F8000A
:10091B00383FFFE0180438003807FFFC1C000000CC
:10092B007801FFFF9C00000078003FFFFC000000F7
:10093B00780007FFFC000000780001FFFC000000BE
:10094B007800003FFC00000078000007FC0000006E
:10095B0078000001FC000000780000003C00000063
:10096B007C000000000000007E0000000000000082
:10097B003F800000000000001FE0000000000000AE
:10098B000FE000000000000003E00000000000008A
:10099B0000E000000000000000000000000000006C
:1009AB00000000000000000000000000000000003C
:1009BB00000000000000000000000000000000002C
:1009CB00000000000000000000000000000000001C
:1009DB00000000000000000000000000000000000C
:1009EB0000000000000000000000000000000000FC
:1009FB0078000000000000007F00000000000000F5
:100A0B00FFC0000000000000FFE00000000000003D
:100A1B00FFE0000000300000F8E00000003FC000E5
:100A2B00F0000000003FF800E00000000001F800BB
:100A3B00E000000000011800E00007F800011800BA
:100A4B00E0000FFE00011800E0001FFF000018007F
:100A5B00F0003FFFC000000070003FFFE000780097
:100A6B0078007FFFE03FF8007C00FFC7F03FF80005
:100A7B003C01FF81F81800003F01FF0078060000E1
:100A8B001FC7FE003C0180000FFFFC003C00E00094
:100A9B000FFFFC001C07F80007FFF8001E3FF800D3
:100AAB0001FFF0000E3F000000FFE0000E0C000005
:100ABB00003FC0000E030000000700001E00C00036
:100ACB000000000C1E0038000000000FFE000800A4
:100ADB000030000FFE30000007FFC00FFE3020007B
:100AEB000FFFF003FC1070001FFFFE00FC00200046
:100AFB003FFFFF00180000007FFFFFC00000000059
:100B0B007FFFFFE000000000FF83FFF80000000004
:100B1B00FE003FFC00000000F80007FE0000000094
:100B2B00F00001FF00300000F000007F803F8000EC
:100B3B00E000001FC00F8000E000000FC0010000AC
:100B4B00E0000007E0018000E0000003F0018000FE
:100B5B00F0000001F008000070000000F83F0000FA
:100B6B0070000000783F8000780000003C2280007D
:100B7B00380000003C2280003C0000001C13800069
:100B8B001C0000001E0300001E0000000E000000F1
:100B9B000F0000000E0180000F0000000E3F8000D0
:100BAB00070000000E3F8000030000000E30000025
:100BBB00000000001E0C0000000000001E060000DC
:100BCB00000000003E01800001FC00187E00800048
:100BDB000FFFC01FFE0000001FFFF01FFC000000F6
:100BEB003FFFFE1FFC0000007FFFFF83FC000000A7
:100BFB007FFFFFC0F8000000FFFFFFF000000000C8
:100C0B00FE03FFF800000000F8003FFC00000000AE
:100C1B00F00007FF00002000F00001FF803E2000E5
:100C2B00E000007FC03FE000E000001FC00FF800B5
:100C3B00E0000007E0003800E0000003F0000000D7
:100C4B00F0000001F000000070000000F800000050
:100C5B007800000078300000780000003C30000085
:100C6B003C0000003C3000003E0000001C00000077
:100C7B001F0000001E3800001F8000000E3C00000B
:100C8B000FE000000E3C780007F000000E22780009
:100C9B0003FC00000E22080001FF00001E210800CB
:100CAB0000FFC0001E210800007FF8003E20F80066
:100CBB00003FFF80FE00F800001FFFFFFE007800E2
:100CCB000007FFFFFC0000000001FFFFFC3C0000E1
:100CDB0000007FFFF83FF00060001FFFF03FF800BF
:100CEB007C0003FFE020F8007F00003F002088001D
:100CFB007FE00000002088007FF80000003C8800A7
:100D0B007FFF0000003FB8003FFFE000001FB8006E
:100D1B0007FFF8001800380001FFFF001800000063
:100D2B00003FFFE0180000000007FFFC1800000068
:100D3B000001FFFF9800000000007FFFF80000009B
:100D4B00000077FFF8000000000071FFFC000000BE
:100D5B000000703FFC00000000007007FC0000006A
:100D6B0000007801FC000000000078003C0000004F
:100D7B00000038001C00000000003C001C000000BC
:100D8B0000003E001C00000000003F001C000000A3
:100D9B0000001F801C00000000001FC03C00000072
:100DAB0000000FF07C000000000007FFFC000000BB
:100DBB00000003FFFC000000700003FFFC000000BC
:100DCB007C0000FFF80000007F00007FF8000000AF
:100DDB007FE0001FF00000003FFC0007E000000078
:100DEB003FFF0000000000003FFFE000000000009C
:100DFB003FFFF8000000000038FFFF001800000064
:100E0B00383FFFE0180000003807FFFC1800000017
:100E1B003801FFFF9800000038003FFFF80000008A
:100E2B0078003FFFFC000000780039FFFC00000059
:100E3B007800383FFC00000078003807FC00000009
:100E4B0078003801FC000000780038003C000000FE
:100E5B007C0038001C0000007E0038001C000000E5
:100E6B003F0038001C0000001FC038001C000000B1
:100E7B000FE038001C00000003E018001C0000000D
:100E8B0000E000001C000000000000001C0000003F
:100E9B000000000E1C0000000000000FFC00000012
:100EAB000000000FFC00000000000007FC00000029
:100EBB0000000001FC000000000000007C000000AE
:100ECB00000000000C00000000000000000000000B
:100EDB000000000000000000000000000000000007
:100EEB007000000000000000700000000000000017
:100EFB0078000000000000007C00000000000000F3
:100F0B007C000000000000007E00000000000000DC
:100F1B007E007800000000007F00FC000000000055
:100F2B007F80FE00000000007FC0FE00000000007C
:100F3B007FC0FF00000000007DE0FF00000000000C
:100F4B007DF00780000000007CF8038000000000AB
:100F5B007CF80180000000007C7C01C000000000D8
:100F6B007C3E01C0000000007C1F83C0000000001D
:100F7B007C1FC3C0000000007C0FFFC000000000FE
:100F8B001807FFC0000000000003FFC000000000B6
:100F9B000001FFC0000000000000FF800000000007
:100FAB00F8003F8000000000FC0000000000000083
:100FBB00FE00000000000000FE000000000000002A
:100FCB00FE000000000000007E000000000000009A
:100FDB003E000000000000000000000000000000C8
:100FEB0000000000000000000000000000000000F6
:100FFB0000000000000000000000000000000000E6
:10100B0000000000000000001FF0000000000000C6
:10101B003FFE0000000000007FFF0000000000000A
:10102B007FFFC00000000000FFFFE0000000000099
:10103B00FFFFF80000000000FC1FF800000000009C
:10104B00F003FC0000000000F000FE0000000000B8
:10105B00E0003F0000000000E0001F000000000067
:10106B00F0000F8000000000F0000780000000007F
:10107B00780003C0000000007C0003C000000000EB
:10108B003E0001C0000000003F0001C00000000056
:10109B001FC003C0000000000FF007C000000000DD
:1010AB0007FF1FC00000000003FFFFC0000000008F
:1010BB0001FFFFC00000000000FFFF8000000000E8
:1010CB00003FFF8000000000000FFF000000000049
:1010DB000001FC0000000000000000000000000008
:1010EB0000000000000000000000000000000000F5
:1010FB00000000FF33FF330000000000000000077A
:10110B00000700000000000700070000002001FEA0
:10111B001FFE1F20012001FE1FFE1F200138063C71
:10112B000E6408FF3FFF3F84091C0F18071E303366
:10113B001C1E07C00170001C1E0733011E1E1FB3AF
:10114B0031E120E120B3311E1F001B803100000074
:10115B000000000B00070000000000000000000072
:10116B0000F807FF3F0738000000000000000000F8
:10117B000000000000000000000000000000000064
:10118B000000000000000000000000000000000054
:10119B000000000000000000000000000000000044
:1011AB000000000000000000000000000000000034
:1011BB000000000000000000000000000000000024
:1011CB000000000030003000000000000000300084
:1011DB003C000FC003F0003C000F000300FC0FFEAF
:1011EB001F0336812161201B30FE1FFC0F042004DE
:1011FB00200620FF3FFF3F0020002000200C380E70
:10120B003C032601238121C3207E203C20061803AA
:10121B00304120412041204120E330BE1F000FE030
:10122B000FFC081F08833F803F000800083F0C3F5E
:10123B001C2130212021206130C11F810FE00FF8CC
:10124B001F5C3046204320C130811F010F0100017C
:10125B00000100013C813FF1037F000F001C0FBE1A
:10126B001FE33041204120E330BE1F1C0F3C207E8A
:10127B0020C32081308118830EFE07FC0100000083
:10128B000000000000000000000000000000000053
:10129B000000000000000000000000000000000043
:1012AB0000000000000000000000000000200120F2
:1012BB00012001200120012001200120010000005C
:1012CB000000000000000000000000000000000013
:1012DB000000000000000000000000000000000003
:1012EB0000000000000000000000000000FC3FFEBA
:1012FB003F0301010101010301FE3FFC3FFF3FFFE3
:10130B003F412041204120E330BE1F1C0FFC0FFE4C
:10131B001F03300120012003300E1C0C0CFF3FFF7C
:10132B003F0120012001200738FE1FF807FF3FFF78
:10133B003F412041204120412041200120FF3FFF20
:10134B003F810081008100810081000100FC0FFEC4
:10135B001F03300120812083308E1F8C0FFF3FFF36
:10136B003F4000400040004000FF3FFF3F01200195
:10137B00200120FF3FFF3F012001200120000C0036
:10138B001C0030002000200030FF1FFF0FFF3FFF2D
:10139B003FC000E00138071C0E0F3C0330FF3FFF3E
:1013AB003F002000200020002000200020FF3FFFF6
:1013BB003F7800C003C0037800FF3FFF3FFF3FFFB4
:1013CB003F1C007000C0010007FF3FFF3F00000003
:1013DB0000000000000000000000000000FF3FFFC5
:1013EB003F810081008100C3007E003C00000000B3
:1013FB0000000000000000000000000000FF3FFFA5
:10140B003F810081008101C31F7E3E3C203C0C7E4E
:10141B001C6330E120C12183318E1F0C0F030003AD
:10142B00000300FF3FFF3F030003000300FF0FFF1C
:10143B001F0030002000200030FF1FFF0F3F00FF78
:10144B0001C00F003C003CC00FFF013F00FF01FF3C
:10145B003F003EC001C001003EFF3FFF0100000006
:10146B000000000000000000000000000000000071
:10147B000000000000000000000000000001380127
:10148B003E8127C121612039201F20072000000049
:10149B000000000000000000000000000000000041
:1014AB000000000000000000000000000000000031
:1014BB000000000000000000000000000000000021
:1014CB000000000000000000000000000000000011
:1014DB000000000000000000000000000000000001
:1014EB0000000000000000000000000000001E4093
:1014FB003F2021202120212011E03FC03FFF3FFF53
:10150B003F4010202020206030C01F800F800FC074
:10151B001F603020202020202060304010800FC022
:10152B001F6030202020204010FF3FFF3F800FC066
:10153B001F6032202220226022C033801320002023
:10154B0000FE3FFF3F21002100230002008007C067
:10155B000F6018201020104008E03FE03F00000013
:10156B000000000000000000000000000000002050
:10157B00202020E33FE33F0020002000000000007C
:10158B0000000000000000000000000000FC3FFC19
:10159B003F00060007800DC01860302020000001BE
:1015AB00200120FF3FFF3F002000200000E03FE034
:1015BB003F6000C01FC01F6000E03FC03FE03FE046
:1015CB003F4000200020006000C03F803F800FC0E4
:1015DB001F6030202020206030C01F800FE03FE0D4
:1015EB003F400420082008600CC007800300000067
:1015FB0000000000000000000000000000E03FE0E1
:10160B003FC00040006000600060004000C010E080
:10161B00312021202320262024603C40180000206C
:10162B00002000FE1FFE3F202020200000E01FE0D6
:10163B003F0020002000200010E03FE03FF003F0CF
:10164B0007001C00300030001CF007F00300000006
:10165B00000000000000000000000000000000007F
:10166B0000000000000000000000000000E001E0AE
:10167B0027002600380018000EE007E0012030207C
:10168B0038202C20262023A021E020602000000001
:10169B00000000000000000000000000000000003F
:1016AB00000000FF3FFF3F000000000000000000B3
:1016BB00000000000000000000000000000000001F
:1016CB00000000000000000000000000000000000F
:1016DB0000000000000000000000000000000000FF
:1016EB0000000000000000000000000000000000EF
:1016FB0000000000000000000000000000000102DC
:10170B00030405060708090A0B0C0D0E0F10111226
:10171B00131415161718191A1B1C1D1E1F20212216
:10172B00232425262728292A2B2C2D2E2F30313206
:10173B00333435363738393A3B3C3D3E3F404142F6
:10174B00434445464748494A4B4C4D4E4F505152E6
:10175B00535455565758595A5B5C5D5E5F000000F9
:10176B00000000000000000000000000000000006E
:10177B00000000000000000000000000000000005E
:10178B00000000000000000000000000000000004E
:10179B00000000000000000000000000000000003E
:1017AB00000000000000000000000000000000002E
:1017BB00000000000000000000000000000000001E
:1017CB00000000000000000000000000000000000E
:1017DB00000000000000000000000000000C000BE7
:1017EB00000A00090008000A000900080031323520
:1017FB006D3F3235306D3F3632356D3F312E3235E0
:10180B003F322E35303F362E32353F31322E353F7B
:10181B0032352E303FFFFF000002000400060008A7
:10182B000012001C0026004E00620076008A009E0B
:10183B0000B200C600EE0016012A013E0166018EC1
:10184B000156021E03E60302000400080035303087
:10185B006E733F312E3075733F322E3075733F33BD
:10186B002E3075733F342E3075733F352E307573B4
:10187B003F31302075733F31352075733F32302047
:10188B0075733F34302075733F35302075733F3699
:10189B00302075733F37302075733F3830207573A8
:1018AB003F39302075733F31303075733F313230F3
:1018BB0075733F31343075733F31353075733F314C
:1018CB00363075733F31383075733F323030757346
:1018DB003F33303075733F34303075733F353030B4
:1018EB0075733F312E306D733F322E306D733F3435
:1018FB002E306D733F3235306E733F3530306E7333
:10190B003F312E3075733F312E3575733F322E308C
:10191B0075733F322E3575733F35202075733F3706
:10192B002E3575733F31302075733F323020757310
:10193B003F32352075733F33302075733F3335207D
:10194B0075733F34302075733F34352075733F35D5
:10195B00302075733F36302075733F3730207573E9
:10196B003F37352075733F38302075733F39302042
:10197B0075733F31303075733F31353075733F328E
:10198B00303075733F32353075733F35303075738A
:10199B003F312E306D733F322E306D733F75B980F2
:1019AB007A14001AEA70FB43B9C0E5B9E5B9A2E5B0
:1019BB0050FA75A90275B28322C082C0831219A88E
:1019CB0075A40D75A5E775A70175D40F75D50775AA
:1019DB00DF0175E10575E242438805E58875E40191
:1019EB00D2A8C2AA759810758D0D538EF4E58E434F
:1019FB008E08858D8B53890FE589438920D28E7490
:101A0B0001901A3EF0D2ACD28C438922E589438EE9
:101A1B000CE58E758CB075C18043E60175D800530B
:101A2B00D9BF75D90275DA4275DB4275FC0775EAC9
:101A3B0007D2DE75C80475CA0175CB01C2ADC2836E
:101A4B00D282D280C292D291D290D2B0C296D2968A
:101A5B00D2AF0228FBD296D282D29275A6FFD29138
:101A6B00C291D291D283C29275A083C280D280D20E
:101A7B009275A002C280D280C283D283C29275A01B
:101A8B0085C280D280D29275A003C280D280C283DD
:101A9B00D283C29275A08CC280D280D29275A09351
:101AAB00C280D280C283D283C29275A091C280D2EF
:101ABB0080D29275A001C280D280C283D283C2929F
:101ACB0075A083C280D280D29275A000C280D280D2
:101ADB00C283D283C29275A03EC280D280D292754D
:101AEB00A0B0C280D280C283D283C29275A03FC203
:101AFB0080D280D29275A003C280D280C283D2835F
:101B0B00C29275A040C280D280D29275A010C280C2
:101B1B00D280C283D283C29275A041C280D280D2BE
:101B2B009275A056C280D280C283D283C29275A016
:101B3B0042C280D280D29275A013C280D280C2835F
:101B4B00D283C29275A043C280D280D29275A04636
:101B5B00C280D280C283D283C29275A044C280D28B
:101B6B0080D29275A023C280D280C283D283C292CC
:101B7B0075A045C280D280D29275A076C280D280E9
:101B8B00C283D283C29275A046C280D280D2927594
:101B9B00A000C280D280C283D283C29275A047C2FA
:101BAB0080D280D29275A05EC280D280C283D28353
:101BBB00C29275A048C280D280D29275A04FC280CB
:101BCB00D280C283D283C29275A049C280D280D206
:101BDB009275A040C280D280C283D283C29275A07C
:101BEB0017C280D280D29275A061C280D280C2838C
:101BFB00D283C29275A02BC280D280D29275A0F9EB
:101C0B00C280D280C283D283C29275A01BC280D203
:101C1B0080D29275A014C280D280C283D283C2922A
:101C2B0075A01AC280D280D29275A011C280D280C8
:101C3B00C283D283C29275A01CC280D280D292750D
:101C4B00A00DC280D280C283D283C29275A01FC264
:101C5B0080D280D29275A03DC280D280C283D283C3
:101C6B00C29275A019C280D280D29275A00AC2808E
:101C7B00D280C283D283C29275A019C280D280D285
:101C8B009275A01AC280D280C283D283C29275A0F1
:101C9B0019C280D280D29275A012C280D280C28328
:101CAB00D283C29275A01EC280D280D29275A02020
:101CBB00C280D280C283D283C29275A03CC280D232
:101CCB0080D29275A060C280D280C283D283C2922E
:101CDB0075A03DC280D280D29275A040C280D280C6
:101CEB00C283D283C29275A034C280D280D2927545
:101CFB00A038C280D280C283D283C29275A035C273
:101D0B0080D280D29275A038C280D280C283D28317
:101D1B00C29275A024C280D280D29275A038C280A4
:101D2B00D280C283D283C29275A024C280D280D2C9
:101D3B009275A03CC280D280C283D283C29275A01E
:101D4B0016C280D280D29275A01CC280D280C28370
:101D5B00D283C29275A001C280D280D29275A006A6
:101D6B00C280D280C283D283C29275A055C280D268
:101D7B0080D29275A000C280D280C283D283C292DD
:101D8B0075A002C280D280D29275A000C280D28090
:101D9B00C283D283C29275A003C280D280D29275C5
:101DAB00A000C280D280C283D283C29275A004C22B
:101DBB0080D280D29275A000C280D280C283D2839F
:101DCB00C29275A005C280D280D29275A0EFC2805C
:101DDB00D280C283D283C29275A006C280D280D237
:101DEB009275A000C280D280C283D283C29275A0AA
:101DFB0007C280D280D29275A000C280D280C283EB
:101E0B00D283C29275A008C280D280D29275A001F3
:101E1B00C280D280C283D283C29275A009C280D203
:101E2B0080D29275A08FC280D280C283D283C2929D
:101E3B0075A022C280D280D292C28375A60075A0F3
:101E4B00FF2275A6FFD283C29275A003C280D280F7
:101E5B00D29289A0C280D280C283D283C29275A053
:101E6B0006C280D280D292EBF5A0C280D280C28310
:101E7B00D283C29275A007C280D280D292EAF5A01B
:101E8B00C280D280C283D283C29275A022C280D27A
:101E9B0080D292C2832274F81202B474081202AA7E
:101EAB00E0FEA3E0FFD283C29275A002C280D28073
:101EBB00D29275A000C280D280C283D283C29275A7
:101ECB00A003C280D280D29289A0C280D280C2836A
:101EDB00D283C29275A004C280D280D29275A00028
:101EEB00C280D280C283D283C29275A005C280D237
:101EFB0080D2928CA0C280D280C283D283C29275D0
:101F0B00A006C280D280D292EBF5A0C280D280C252
:101F1B0083D283C29275A007C280D280D292EAF597
:101F2B00A0C280D280C283D283C29275A008C28025
:101F3B00D280D292EFF5A0C280D280C283D283C26C
:101F4B009275A009C280D280D292EEF5A0C280D247
:101F5B0080C283D283C29275A022C280D280D292D9
:101F6B00C2830222F874F71202B474091202AAE0B7
:101F7B00F508A3E0F5097E987F9E75A6FF780812F9
:101F8B00034C121EA17402120275D283C29275A069
:101F9B0022C280D280D292C283901047E0FAA3E093
:101FAB00D283F5A0C280D280EAF5A0C280D280C2D3
:101FBB0083901047E0FAA3E0D283F5A0C280D280D1
:101FCB00EAF5A0C280D280C283EEF8EFF974FF2845
:101FDB001E74FF39FFE87001E970BE75088F750933
:101FEB0001780812034C7CEF7A007B007900121EFB
:101FFB00A1740212027502453474F81202B4EAFE9F
:10200B00EBFFD29675A6FF7A007B007900121E4D6E
:10201B00D283C29275A022C280D280D292C2837A1E
:10202B00F97BC0EFFCD2838CA0C280D280EEF5A0EE
:10203B00C280D280C283D2838CA0C280D280F5A012
:10204B00C280D280C283EA1A70DBEB1B70D70222EC
:10205B00F874F41202B4890BEC24E8F582E434161C
:10206B00F583E493901044F0F50875090074037838
:10207B000812024C901042E508F0A3E509F08A081B
:10208B008B09901042E0F8A3E0F9E8C333F8E93389
:10209B00F9E824E8FEE93410FF750A08AA08AB0931
:1020AB00A90B121E4D78007920D283C29275A02203
:1020BB00C280D280D292C283750C0E8E828F83E443
:1020CB009358FAA3E49359FBEA7001EB6005901067
:1020DB00458003901047E0FCA3E0D283F5A0C280BB
:1020EB00D280ECF5A0C280D280C283E9C313F9E899
:1020FB0013F8150CE50C70C3EE24020E0EEF340032
:10210B00FFE5082401F508E5093400F509150AE592
:10211B000A708902444474F11202B4890AECFEED90
:10212B008A0C8B0D750838750906750E56750F01DF
:10213B00F50BAA0CAB0DA90A121E4DD283C29275D8
:10214B00A022C280D280D292C28385088285098365
:10215B007B087C807A08E4935CD283600C850BA0AF
:10216B00C280D280EEF5A0800A75A074C280D280A6
:10217B0075A053C280D280C283ECC313FC1AEA70E1
:10218B00D5A31BEB70CCE5082408F508E509340052
:10219B00F509E50C2401F50CE50D3400F50DE50E04
:1021AB0024FFF50EE50F34FFF50FE50E7002E50F7A
:1021BB0070808004C296D2967F0802031474F812C2
:1021CB0002B4901047E4F0A3F090104974BFF0A351
:1021DB00741DF090104574FFF0A3F0901047E0FAD7
:1021EB00A3E0FB12200490103EE0D2E0F07C8F7D48
:1021FB00017A017B0079121222FD7C8F7D017A011D
:10220B007B0079011222FD7C8F7D017A017B0079A5
:10221B00DF1222FD7C8F7D017A017B0079EF122288
:10222B00FD7E007F007582747583198019EEFAEFBD
:10223B00FBEA75F00AA4FAADF075F00AEBA42DFBDE
:10224B00790212205CA3E0FAEE24010EEF3400FFBA
:10225B00EAFC743F6A70D67E007F0075829C7583A2
:10226B00198019EEFAEFFBEA75F00AA4FAADF075D6
:10227B00F00AEBA42DFB79E112205CA3E0FAEE242B
:10228B00010EEF3400FFEAFC743F6A70D6901045E4
:10229B0074E6F0A374FFF07582C27583197EC87F54
:1022AB00008012EEFAEFFB790212205CEE240AFE9C
:1022BB00EF3400FFA3E0FAFC743F6A70E690104520
:1022CB0074BFF0A3741DF07582C27583197E2C7FC9
:1022DB00018012EEFAEFFB790212205CEE240AFE6B
:1022EB00EF3400FFA3E0FAFC743F6A70E67F010253
:1022FB00031474F61202B4890A8A088B09ECFEEDFA
:10230B00FF121E4D90103EE0A2E0E492E012035D3E
:10231B0000018E2323234F23901049E0FAA3E0D230
:10232B0083F5A0C280D280EAF5A0C280D280C2839E
:10233B00EEF8EFF974FF281E74FF39FFE87001E91E
:10234B0070D6803F901049E0FAA3E0D283F5A0C28B
:10235B0080D280EAF5A0C280D280C283AA08AB09E2
:10236B00A90A121E4DE5082401F508E5093400F50C
:10237B0009EEF8EFF974FF281E74FF39FFE87001BE
:10238B00E970C17F0302031474F71202B490104971
:10239B0074EFF0A3747BF07508197509007E147F38
:1023AB0000AA08AB09EEF9121E4D901049E0FAA3F2
:1023BB00E0D283F5A0C280D280EAF5A0C280D280A1
:1023CB00C283EE2405FEEF3400FFC3EE94E0EF94DE
:1023DB000040CEE5082419F508E5093400F509C3DA
:1023EB00E508948FE509940140B37508147509004D
:1023FB007E007F00EEFAEFFBA908121E4D901049EC
:10240B00E0FAA3E0D283F5A0C280D280EAF5A0C2A5
:10241B0080D280C283EE2405FEEF3400FFC3EE941E
:10242B008FEF940140CEE5082419F508E509340037
:10243B00F509C3E50894E0E509940040B390103E1C
:10244B00E0C2E0F07CC87D007AC87B0079141222D0
:10245B00FDE0D2E0F07C8F7D017A007B0079781271
:10246B0022FD02453474F51202B4901049E0F50ACE
:10247B00A3E0F50B901049E4F0A3F0901047F0A304
:10248B00F090103EE0C2E0F07E127F007508297CD0
:10249B000D7D00EEFAEFFB79021222FD7C0D7D0023
:1024AB0074012EFAE43FFB79021222FDEE240AFEA0
:1024BB00EF3400FF1508E50870D5E0C2E0F07E129E
:1024CB007F007508297C0D7D00EEFAEFFB79E11298
:1024DB0022FD7C0D7D0074012EFAE43FFB79E112A5
:1024EB0022FDEE240AFEEF3400FF1508E50870D537
:1024FB0090104574E6F0A374FFF07E007F00750822
:10250B00BE8E098015AA08AB09790212205CE5087A
:10251B00240AF508E5093400F509EE24EEF582EFFF
:10252B003419F583E0FAEE24010EEF3400FFEAFCD8
:10253B00743F6A70D090104574BFF0A3741DF07E89
:10254B00007F007508227509018015AA08AB09796F
:10255B000212205CE508240AF508E5093400F509A8
:10256B00EE24F8F582EF3419F583E0FAEE24010E30
:10257B00EF3400FFEAFC743F6A70D090103CE0A28D
:10258B00E7901045500874E0F0A37407800474FFC3
:10259B00F0A3F07E007F0075085A8E098015AA08FB
:1025AB00AB0979E112205CE508240AF508E509344A
:1025BB0000F509EE240CF582EF341AF583E0FAEE00
:1025CB0024010EEF3400FFEAFC743F6A70D09010C8
:1025DB0000E0700B90104574E6F0A374FF80136459
:1025EB0001901045700874BFF0A3741D800474FF34
:1025FB00F0A3F07E007F0075085A8E098015AA089B
:10260B00AB09790212205CE508240AF508E50934C8
:10261B0000F509EE24E4F582EF3419F583E0FAEEC8
:10262B0024010EEF3400FFEAFC743F6A70D0901067
:10263B004574FFF0A3F07E007F007508148E0980AF
:10264B0015AA08AB09790212205CE508240AF508E3
:10265B00E5093400F509EE24DAF582EF3419F58338
:10266B00E0FAEE24010EEF3400FFEAFC743F6A70CF
:10267B00D07E007F007508148E098015AA08AB095F
:10268B0079E112205CE508240AF508E5093400F528
:10269B0009EE2402F582EF341AF583E0FAEE2401F9
:1026AB000EEF3400FFEAFC743F6A70D07E007F00AF
:1026BB007508968E098015AA08AB0979E112205C82
:1026CB00E508240AF508E5093400F509EE2416F5AA
:1026DB0082EF341AF583E0FAEE24010EEF3400FF9B
:1026EB00EAFC743F6A70D07E007F007508E68E09A5
:1026FB008015AA08AB0979E112205CE508240AF5DC
:10270B0008E5093400F509EE2420F582EF341AF5BB
:10271B0083E0FAEE24010EEF3400FFEAFC743F6A0B
:10272B0070D07E007F007508367509018015AA08E8
:10273B00AB0979E112205CE508240AF508E50934B8
:10274B0000F509EE242AF582EF341AF583E0FAEE50
:10275B0024010EEF3400FFEAFC743F6A70D0901036
:10276B0049E50AF0A3E50BF07F04020314C082C015
:10277B0083740190102FF090103FE04412F07959C0
:10278B001228749019D8E090101BF090102FE09045
:10279B00101CF0901030E090101DF0901031E09074
:1027AB00101EF0740290102FF090103FE04412F0C6
:1027BB00795912287490102FE090101FF090103060
:1027CB00E0901020F0901031E0901021F074089000
:1027DB00102FF090103FE04412F0795912287490AA
:1027EB00102FE0901022F0901030E0901023F0901A
:1027FB001031E0901024F0740E90102FF090103FD9
:10280B00E0C2E1F0D2E4F0795912287490102FE075
:10281B00901025F0901030E0901026F07437901047
:10282B002FF090103FE0C2E1F0D2E4F0795912287A
:10283B007490102FE0901027F0901030E09010283B
:10284B00F0740D90102FF090103FE0C2E1F0D2E445
:10285B00F0795912287490102FE0901029F09010F5
:10286B0030E090102AF00228FBC082C0837A007BF4
:10287B000090103FA2A8E092E3F0C2A8E99019D80B
:10288B00F090103FE0D2E0F0A2E45007C2E4F0D2A7
:10289B00E28002C2E2F0D2C5E0A2E0501BEAF8EB04
:1028AB00F97401280AE439FBC3E89441E9949C408C
:1028BB00ECE0C2E0F0C340E5901041E0A2E250280A
:1028CB00E0A2E14023E4901030F0901031F074015D
:1028DB0090102FF090103FE0C2E2F0D2C5A2E04082
:1028EB00FC901041E0C2E2F090103FE0A2E392A80E
:1028FB00D083D08222C0E0C0D0E8C0E0E9C0E0EADB
:10290B00C0E0C082C083A2984003022AA990103F66
:10291B00E0A2E05016901018E0FA74012AF0EAC316
:10292B009415400C90103FE0C2E0F0E4901018F0CA
:10293B00901011E07007901014E4F0A3F0C298E52A
:10294B009990101AF0901011E0C394114003022AD1
:10295B00A990101AE0C0E0901014E02401F8A3E055
:10296B003410F988828983D0E0F0901011E004F0E4
:10297B00901014E02401F0A3E03400F0901011E06B
:10298B0064106003022AA9901010E0640D6003022A
:10299B002A9190103CC082901001E0A2E075831048
:1029AB00D082E092E3F090103CC082901002E0A243
:1029BB00E0758310D082E092E1F090103CC08290E1
:1029CB001003E0A2E0758310D082E092E2F0901049
:1029DB003CE0A2E1400DE0A2E24008901004E09040
:1029EB001036F0901005E0901030F0901006E0904B
:1029FB001031F0901007E090102FF0901008E0903D
:102A0B0019D8F0901009E09019D9F090100AE090C5
:102A1B001019F090103CC08290100BE0A2E075836F
:102A2B0010D082E092E6F0901019E064017004C2BD
:102A3B00B08002D2B090103CE0A2E3E05014E0C2B0
:102A4B0096901034E4F0A3F0D29690103CE0C2E0E4
:102A5B00800CA2E140F7E0A2E240F2E0D2E0F0907D
:102A6B00102FE06401700890103FE0D2E18010E07D
:102A7B00640260F3E0640860EE90103FE0C2E1F0A6
:102A8B00E49010118017E4901011F090103CE0D2FC
:102A9B00E0F0E0C2E3F0E0C2E1F0E0C2E2F0A299C4
:102AAB005056C2999019D6E07002A3E0603A901983
:102ABB00D6E0F8A3E0F9901012E0687003A3E06988
:102ACB007007901016E4F0A3F090101AE0F59990AF
:102ADB001016E02401F0A3E03400F09019D6E024A6
:102AEB00FFF0A3E034FF800F901012E0F8A3E0F9A1
:102AFB009019D6E8F0A3E9F0D083D082D0E0FAD0D9
:102B0B00E0F9D0E0F88004D083D082D0D0D0E0328E
:102B1B00C0E0C0D0C082C083C0F0A2C25003022C60
:102B2B001B74F055C01203D9000380E02BC05D2B42
:102B3B00E0402B1B2C9019D8E0C333F5C253C2FED7
:102B4B0090103FE0A2E4E492E045C2F5C2C2C50298
:102B5B002C1BA2C1506E90103FE0A2E45003022C3C
:102B6B001BA2E14008901032E064026047901032E3
:102B7B00E012035D00031B2C8B2B9A2BB42BBF2B6A
:102B8B00901032E004F090102FE0F5C2022C1B9055
:102B9B00103FE0A2E25007D2E4F0D2C58072901051
:102BAB0032E004F090103080E0901032E004F090AE
:102BBB00103180D590103FE0C2E0F0E4901032F07D
:102BCB00D2C4804CE4901032F0D2C49019D8E06497
:102BDB005D603D80C5901032E012035D01011B2C3E
:102BEB00EF2B072CE5C2901030F0901032E004F080
:102BFB0090103FE0A2E1500AD2C18014E5C29010C0
:102C0B0031F0C2C1E4901032F090103FE0C2E0F01E
:102C1B00C2C0D0F0022B12C0E0C0D0C082C083D2A1
:102C2B009090103CE0D2E4F0022B12C0E0C0D0EA4E
:102C3B00C0E0C082C083901A3FE0FA74012AF0EA28
:102C4B00C39405405C75A60075A0FFC296C2839025
:102C5B001040A2A5E092E0F0A2A0E092E1F0A2A6C3
:102C6B00E092E2F0A2A7E092E3F0A2A2E092E4F0FD
:102C7B00A2A1E092E5F0A2A3E092E6F0A2A4E0927A
:102C8B00E7F0E064FF6013901041E0A2E4400BE03A
:102C9B00D2E3F090103CE0C2E3F0D296E4901A3FFE
:102CAB00F0C2CFD083D082D0E0FA022B16C2AD9007
:102CBB001041E0D2E4F074FF901040F074029010D9
:102CCB0000F090103DE0D2E0F0E0D2E1F0D2B01293
:102CDB0019C47418901030F07440901031F07402D5
:102CEB0090102FF0901041E0D2E2F090103FE0C234
:102CFB00E4F0D2E1F0901041E0C2E1F079591228F2
:102D0B0074E0D2E2F07403901033F090103FE05473
:102D1B00EDF0740390102FF0795D12287490103F32
:102D2B00E054EDF0740890102FF07948122874904D
:102D3B00103FE054EDF0740890102FF079491228F1
:102D4B0074121A6075A6FF7A537B741220049010CC
:102D5B00457437F0A374FFF09010477453F0A374CD
:102D6B0074F07C377DFF7A237B00795A1221217511
:102D7B00824E7583197E1E7F008012EEFAEFFB796F
:102D8B001912205CEE240AFEEF3400FFA3E0FAFCDC
:102D9B00743F6A70E6D2AD901040E064FF60F8902B
:102DAB001041E0C2E4F0C2AD1221C812239390107F
:102DBB003CE0D2E5F0E0D2E3800EC296D296122F21
:102DCB001DE0C2E3F0E0D2E0F0E0A2E54057E0A264
:102DDB00E040FBE0A2E340E2E0A2E1501F122778C3
:102DEB009019D67414F0A3E4F09010127414F0A39D
:102DFB00E4F0D29990103CE0C2E180C8E0A2E2502E
:102E0B00C890103FE0C2E4F09019D8E0F912287492
:102E1B007401901A3EF090103CE0C2E280A612279B
:102E2B0078E0C2E1F090103CE0A2E54003022F1CD9
:102E3B00800AE0A2E15005C2AD12359ED2AD9010D2
:102E4B003CE0A2E3E0502FA2E75007C2AD123A33A9
:102E5B0080EA90103DE0FAE0FBEAA2E0500CEBA216
:102E6B00E15007C2AD12371D80D2E0A2E050C3C2C1
:102E7B00AD12341D80C6A2E140A4E0A2E250219025
:102E8B00103FE0C2E4F09019D8E0F91228747401F5
:102E9B00901A3EF090103CE0C2E2F0E0D2E3808466
:102EAB00901041E0A2E34003022E3090103CE0C2B0
:102EBB00E2F0901040E0A2E2401B901033E0640877
:102ECB00F090103FE054EDF0901033E090102FF0A5
:102EDB00795D122874901040E0A2E3401B901033F0
:102EEB00E06410F090103FE054EDF0901033E09060
:102EFB00102FF0795D122874C2AD123BE490104193
:102F0B00E0C2E3F090103CE0A2E25003022E3080CE
:102F1B008A22C082C083D2A8C29090103CE0A2E467
:102F2B0050F8E0C2E4F0C2A8D290901036E06004F2
:102F3B0064027033901034E4F0A3F0D297C297D2AE
:102F4B0097901034E02401F0A3E03400F09010349B
:102F5B00C3E094FFA3E0940140E1D297901012E4F8
:102F6B00F0A37402F0D299901019E064016005E0AF
:102F7B006402700890103CE0A2E650F8901036E026
:102F8B0064016005E064027031901034E4F0A3F04A
:102F9B00D295C295D295901034E02401F0A3E03481
:102FAB0000F0901034C3E094FFA3E0940140E19053
:102FBB001012E4F0A37402F0D299C296D2960228B2
:102FCB00FB74F51202B47E00E4901947F075A6006D
:102FDB0075A0FF786B79137A10C297E5A02438F5AA
:102FEB0082E43404F583E49388828983F0A3E4F0CC
:102FFB00D297E824020808E93400F91AEA70DA7F5C
:10300B0008787B7913C297E82410FAE93400FBE5C2
:10301B00A02438F582E43404F583E4938A828B830D
:10302B00F0A3E4F0D297EE705B901A40E0F50888BD
:10303B00828983E0FCA3E0FD74FC2508F50A74FF8C
:10304B003400F50BC3E50A9CE50B9DA2D265D0338A
:10305B00503274042508F508E43400F509EC9508A2
:10306B00ED9509A2D265D033501A8A828B83E0FA90
:10307B00C3EC9AED9400A2D265D0335007EF9019B0
:10308B0047F07E010FE824020808E93400F9EFC38A
:10309B00945C500302301002277374F41202B4755F
:1030AB000A00E4901947F075A60075A0FF785379D4
:1030BB00177A10C295E5A02438F582E43404F58321
:1030CB00E49388828983F0D295A3A882A9831AEA14
:1030DB0070E1750B08785B7917C295E82408FAE95B
:1030EB003400FBE5A02438F582E43404F583E49343
:1030FB008A828B83F0D295E50A704E88828983E0B1
:10310B00F582AE82901A40E0FC74FC2CF50874FF3B
:10311B003400F509C3E5089EE5099400A2D265D0F9
:10312B0033502674042CFCE43400FDEE9CE49DC368
:10313B0065D03350148A828B83E0FAEEC39A500920
:10314B00E50B901947F0750A01050B88828983A35B
:10315B00A882A983E50BC3945C50030230E40244BC
:10316B004474F21202B47E00E4901947F075A60085
:10317B0075A0FF7A537B17786B79137C10C297E598
:10318B00A02438F582E43405F583E493F5088882AE
:10319B008983F0A3E4F0D297C295E5A02438F58299
:1031AB00E43405F583E4938A828B83F0D295E8248B
:1031BB00020808E93400F9A3AA82AB831CEC70BDAA
:1031CB007F087C5B7D177A7B7B13C297EA2410F810
:1031DB00EB3400F9880A890BE5A02438F582E43436
:1031EB0005F583E49388828983F0A3E4F0D297C238
:1031FB0095EC2408F8ED3400F9880C890DE5A02432
:10320B0038F582E43405F583E49388828983F0D220
:10321B0095EE60030232DE901000E07065901A406C
:10322B00E0F88A828B83E0F508A3E0F50974FC28AB
:10323B00F50C74FF3400F50DC3E50C9508E50D9501
:10324B0009A2D265D03340030232DE740428F8E4BD
:10325B003400F9E50898E50999A2D265D03350738B
:10326B00850A82850B83E0F8A3E0F9C3E50898E5AE
:10327B000999A2D265D033505AEF901947F07E01CD
:10328B0080516401704D8C828D83E0F50EF5828543
:10329B008208901A40E0F874FC28F50A74FF340099
:1032AB00F50BC3E50A9508E50B9400A2D265D03364
:1032BB005021740428F8E43400F9E50898E499C324
:1032CB0065D033500E850C82850D83E0F8E50EC377
:1032DB009840A60FEA24020A0AEB3400FB8C828D7D
:1032EB0083A3AC82AD83EFC3945C50030231D57FD3
:1032FB000702031474F51202B47E00E4901947F030
:10330B0075A60075A0FF786B79137A08C297E5A0B4
:10331B002438F582E43404F583E49388828983F0BE
:10332B00A3E4F0D297C295E5A02438F582E43404E7
:10333B00F583E49388828983A3A3F0A3E4F0D29569
:10334B00E82404F8E93400F91AEA70C07F08787BA6
:10335B007913C297E82410FAE93400FBE5A024386E
:10336B00F582E43404F583E4938A828B83F0A3E43F
:10337B00F0D297C295E5A02438F582E43404F583A6
:10338B00E493FCE82412F582E93400F583ECF0A316
:10339B00E4F0D295EE7065901000E06402605D90F1
:1033AB001A40E0F50888828983E0FCA3E0FD74FCF9
:1033BB002508F50A74FF3400F50BC3E50A9CE50BF1
:1033CB009DA2D265D033503474042508F508E4343B
:1033DB0000F509EC9508ED9509A2D265D033501C88
:1033EB008A828B83E0FAA3E0FBC3EC9AED9BA2D21B
:1033FB0065D0335007EF901947F07E010F0FE8248B
:10340B0004F8E93400F9EFC3945B500302335D0217
:10341B00277374F11202B4D2A8C29090103CE0A2B0
:10342B00E450F8E0C2E4F0C2A8122FCC901000E0F8
:10343B00640270087401901947F08009901947E0F5
:10344B00700302359B7E007F0075084B7509107564
:10345B000E33750F14E0C333F8E433F9E8246BF53E
:10346B000CE93413F50D75A60075A0FFC297E5A006
:10347B002438F582E43404F583E493850E82850FBA
:10348B0083F0A3E4F0D29775A6FF850882850983A4
:10349B00E0FC74786C600874C86E7001EF700B9070
:1034AB00104974EFF0A3747B8052EC75F00584E542
:1034BB00F07011EEF8EFF97A197B001201E3EA7064
:1034CB0001EB60DB8C0A7405250AF8E43400F97A09
:1034DB00197B001201DBEA7001EB7011EEF8EFF9CA
:1034EB007A057B001201E3EA7001EB60B2901047A2
:1034FB00E0F8A3E0F9901049E8F0A3E9F0EEFAEF59
:10350B00FBECF9121E4D901049E0FAA3E0D283F5C3
:10351B00A0C280D280EAF5A0C280D280C283901074
:10352B004974E6F0A374FFF0850C82850D83E024CB
:10353B00F8F50AEEFAEFFBA90A121E4D901049E0BE
:10354B00FAA3E0D283F5A0C280D280EAF5A0C280B4
:10355B00D280C283850882850983E50AF0EE2401B7
:10356B000EEF3400FFE50C2402F50CE50D3400F5ED
:10357B000DE50E2402F50EE50F3400F50FA3858241
:10358B0008858309C3EE948FEF94015003023471C5
:10359B000221BF74F11202B4D2A8C29090103CE089
:1035AB00A2E450F8E0C2E4F0C2A81230A5901000DB
:1035BB00E0640270087401901947F0800990194774
:1035CB00E0700302371A7E007F00750EB7750F1778
:1035DB007508DB750911E02453F50CE43417F50D70
:1035EB0075A60075A0FFC295E5A02438F582E434DA
:1035FB0004F583E493850E82850F83F0D29575A62F
:10360B00FF850882850983E0FC74786C600874C8B8
:10361B006E7001EF700B90104974EFF0A3747B8008
:10362B0052EC75F00584E5F07011EEF8EFF97A19AC
:10363B007B001201E3EA7001EB60DB8C0A74052559
:10364B000AF8E43400F97A197B001201DBEA700105
:10365B00EB7011EEF8EFF97A057B001201E3EA70DB
:10366B0001EB60B2901047E0F8A3E0F9901049E845
:10367B00F0A3E9F0EEFAEFFBECF9121E4D901049B6
:10368B00E0FAA3E0D283F5A0C280D280EAF5A0C213
:10369B0080D280C28390104974BFF0A3741DF08553
:1036AB000C82850D83E024F8F50AEEFAEFFBA90AEC
:1036BB00121E4D901049E0FAA3E0D283F5A0C28010
:1036CB00D280EAF5A0C280D280C2838508828509A8
:1036DB0083E50AF0EE24010EEF3400FF850C8285A2
:1036EB000D83A385820C85830D850882850983A3B1
:1036FB00858208858309850E82850F83A385820EBB
:10370B0085830FC3EE948FEF940150030235EB02C8
:10371B0021BF74F11202B474FA12025FD2A8C290E4
:10372B0090103CE0A2E450F8E0C2E4F0C2A81231E1
:10373B006C901000E0640270087401901947F080DF
:10374B0009901947E07003023A277E007F0074044A
:10375B001202AA74B7F0A37417F0750C4B750D1009
:10376B007508DB750911901947E0F82453FAE43416
:10377B0017FB74021202AAEAF0A3EBF08510828504
:10378B0011837433F0A37414F0E8C333F8E433F902
:10379B00E8246BF50EE93413F50F75A60075A0FF41
:1037AB00C297E5A02438F582E43405F583E493FA57
:1037BB00851082851183E0F8A3E0F5838882EAF017
:1037CB00A3E4F0D297C295E5A02438F582E4340542
:1037DB00F583E493C0E074041202AAE0F8A3E0F5C9
:1037EB00838882D0E0F0D29575A6FF850C82850D7B
:1037FB0083E0FC74786C600874C86E7001EF700B1A
:10380B0090104974EFF0A3747B8052EC75F0058433
:10381B00E5F07011EEF8EFF97A197B001201E3EA8B
:10382B007001EB60DB8C0A7405250AF8E43400F9AF
:10383B007A197B001201DBEA7001EB7011EEF8EFE5
:10384B00F97A057B001201E3EA7001EB60B290108C
:10385B0047E0F8A3E0F9901049E8F0A3E9F0EEFA9D
:10386B00EFFBECF9121E4D901049E0FAA3E0D28366
:10387B00F5A0C280D280EAF5A0C280D280C2838537
:10388B000882850983E0FC74786C600874C86E70DC
:10389B0001EF700B90104974EFF0A3747B8052EC26
:1038AB0075F00584E5F07011EEF8EFF97A197B00ED
:1038BB001201E3EA7001EB60DB8C0A7405250AF850
:1038CB00E43400F97A197B001201DBEA7001EB702A
:1038DB0011EEF8EFF97A057B001201E3EA7001EBC8
:1038EB0060B2901047E0F8A3E0F9901049E8F0A31C
:1038FB00E9F0EEFAEFFBECF9121E4D901049E0FAED
:10390B00A3E0D283F5A0C280D280EAF5A0C280D218
:10391B0080C28390104974E6F0A374FFF0850E8289
:10392B00850F83E0246AF50AEEFAEFFBA90A121E53
:10393B004D901049E0FAA3E0D283F5A0C280D2806B
:10394B00EAF5A0C280D280C283850C82850D83E507
:10395B000AF090104974BFF0A3741DF074021202A8
:10396B00AAE0F8A3E0F5838882E02406F50AEEFAD4
:10397B00EFFBA90A121E4D901049E0FAA3E0D28387
:10398B00F5A0C280D280EAF5A0C280D280C2838526
:10399B000882850983E50AF0EE24010EEF3400FF5F
:1039AB00E50E2402F50EE50F3400F50F8510828528
:1039BB001183E02402F8A3E03400F985108285110D
:1039CB0083E8F0A3E9F074021202AAE02401F8A341
:1039DB00E03400F974021202AAE8F0A3E9F08508BA
:1039EB0082850983A3858208858309850C82850DD1
:1039FB0083A385820C85830D74041202AAE0240133
:103A0B00F8A3E03400F974041202AAE8F0A3E9F079
:103A1B00C3EE948FEF940150030237A5C296D29652
:103A2B0074061202750221C374F31202B4D2A8C237
:103A3B009090103CE0A2E450F8E0C2E4F0C2A8126F
:103A4B0032FF901000E0640270087401901947F087
:103A5B008009901947E07003023BDB75A60075A047
:103A6B00FF7E007F0078337914C297E5A02438F5E8
:103A7B0082E43404F583E49388828983F0A3E4F031
:103A8B00D297C295E5A02438F582E43404F583E49B
:103A9B009388828983A3A3F0A3E4F0D295EE24024A
:103AAB000E0EEF3400FFE82404F8E93400F9C3EEFE
:103ABB00948EEF940140B275A6FF7E007F007508CF
:103ACB004B750910901947E0C333F8E433F9E82438
:103ADB006BF50CE93413F50D850882850983E0FC41
:103AEB0074786C600874C86E7001EF700B9010499D
:103AFB0074EFF0A3747B8052EC75F00584E5F070E5
:103B0B0011EEF8EFF97A197B001201E3EA7001EB81
:103B1B0060DB8C0A7405250AF8E43400F97A197B0A
:103B2B00001201DBEA7001EB7011EEF8EFF97A0588
:103B3B007B001201E3EA7001EB60B2901047E0F8F2
:103B4B00A3E0F9901049E8F0A3E9F0EEFAEFFBECF3
:103B5B00F9121E4D901049E0FAA3E0D283F5A0C2F2
:103B6B0080D280EAF5A0C280D280C28390104974C3
:103B7B00FFF0A3F0850C82850D83E024F8F50AEEA7
:103B8B00FAEFFBA90A121E4D901049E0FAA3E0D2FE
:103B9B0083F5A0C280D280EAF5A0C280D280C28316
:103BAB00850882850983E50AF0EE24010EEF3400C7
:103BBB00FFE50C2402F50CE50D3400F50DA3858211
:103BCB0008858309C3EE948FEF94015003023AE307
:103BDB00C296D2967F0602031474F41202B49010AC
:103BEB0049E0F50AA3E0F50B901049E4F0A374F853
:103BFB00F0901040E0A2E7E492E044FEF4FA90105B
:103C0B0037E02AF0901040E0A2E6E492E044FEF4A4
:103C1B00FA901037E0C39AF064FF705D7409F012EC
:103C2B00247090103EE0C2E0F07E347F01750806F0
:103C3B007C0D7D00EEFAEFFB79E11222FD7C0D7D10
:103C4B000074012EFAE43FFB79E11222FDEE240A07
:103C5B00FEEF3400FF1508E50870D5901047E4F02F
:103C6B00A374F8F090104574FFF0A3F07E007F0072
:103C7B007508367509010243F5E0C3940A4004E464
:103C8B00F0801CE012035D00093344AA3CB33C3EB8
:103C9B003DD33D653EF53E833F7E422F432A3C128A
:103CAB00444912247002443312247090103EE0C237
:103CBB00E0F07E127F007508077C0D7D00EEFAEFB9
:103CCB00FB79021222FD7C0D7D0074012EFAE43F7C
:103CDB00FB79021222FDEE240AFEEF3400FF1508D9
:103CEB00E50870D5901047E4F0A374F8F0901045F8
:103CFB0074FFF0A3F07E007F007508148E09EE248C
:103D0B00DAF582EF3419F583E0FAEE24010EEF3485
:103D1B0000FFEAFC743F6A7003024275AA08AB0904
:103D2B00790212205CE508240AF508E5093400F550
:103D3B000980CB12247090103EE0C2E0F07E587FD9
:103D4B000075080A7C0D7D00EEFAEFFB790212225A
:103D5B00FD7C0D7D0074012EFAE43FFB79021222EB
:103D6B00FDEE240AFEEF3400FF1508E50870D59030
:103D7B001047E4F0A374F8F090104574FFF0A3F033
:103D8B007E007F0075085A8E098015AA08AB097949
:103D9B000212205CE508240AF508E5093400F50950
:103DAB00EE24E4F582EF3419F583E0FAEE24010EEC
:103DBB00EF3400FFEAFC743F6A70D0901047E4F0D8
:103DCB00A3F012453902443312247090103EE0C226
:103DDB00E0F07EBC7F0075080A7C0D7D00EEFAEFEB
:103DEB00FB79021222FD7C0D7D0074012EFAE43F5B
:103DFB00FB79021222FDEE240AFEEF3400FF1508B8
:103E0B00E50870D5901047E4F0A374F8F0901045D6
:103E1B0074E6F0A374FFF07E007F007508BE8E0978
:103E2B008015AA08AB09790212205CE508240AF573
:103E3B0008E5093400F509EE24EEF582EF3419F5A7
:103E4B0083E0FAEE24010EEF3400FFEAFC743F6AC4
:103E5B0070D0790012485B02443312247090103EEC
:103E6B00E0C2E0F07E207F0175080A7C0D7D00EE3C
:103E7B00FAEFFB79021222FD7C0D7D0074012EFA04
:103E8B00E43FFB79021222FDEE240AFEEF3400FF21
:103E9B001508E50870D5901047E4F0A374F8F0907E
:103EAB00104574BFF0A3741DF07E007F00750822CF
:103EBB007509018015AA08AB09790212205CE50887
:103ECB00240AF508E5093400F509EE24F8F582EF2C
:103EDB003419F583E0FAEE24010EEF3400FFEAFC0F
:103EEB00743F6A70D07901023E5F12247090103ECD
:103EFB00E0C2E0F07E127F007508077C0D7D00EEBE
:103F0B00FAEFFB79E11222FD7C0D7D0074012EFA94
:103F1B00E43FFB79E11222FDEE240AFEEF3400FFB1
:103F2B001508E50870D5901047E4F0A374F8F090ED
:103F3B00104574FFF0A3F07E007F007508148E0906
:103F4B008015AA08AB0979E112205CE508240AF573
:103F5B0008E5093400F509EE2402F582EF341AF571
:103F6B0083E0FAEE24010EEF3400FFEAFC743F6AA3
:103F7B0070D01247A602443312247090103EE0C258
:103F8B00E0F07E587F007508067C0D7D00EEFAEFA1
:103F9B00FB79E11222FD7C0D7D0074012EFAE43FCA
:103FAB00FB79E11222FDEE240AFEEF3400FF150827
:103FBB00E50870D5901047E4F0A374F8F090104525
:103FCB0074FFF0A3F07E007F0075085A8E098015F0
:103FDB00AA08AB0979E112205CE508240AF508E58B
:103FEB00093400F509EE240CF582EF341AF583E061
:103FFB00FAEE24010EEF3400FFEAFC743F6A70D036
:10400B0090103CE0A2E740030240F4901040E0A285
:10401B00E550030241D790103CE0C2E7F090104707
:10402B00E4F0A3F075088F750901780812034C7C36
:10403B00DE7A007B007914121F7074021202751263
:10404B0023937E487F1990103AE0F8A3E0F9E875C6
:10405B00F006A4F8AAF075F006E9A42AF9E82458AA
:10406B00FAE93418FBEAF8EBF97CDA7D19750805E7
:10407B0088828983E493F5098E828F83F0EC240B7D
:10408B00F582ED3400F583E509F08C828D83A3ACCA
:10409B0082AD8388828983A3A882A9838E828F8332
:1040AB00A3AE82AF831508E50870C58A828B83A304
:1040BB00A3A3A3A3E49390194DF0901047E4F0A3AE
:1040CB00F07582487583197E64FFE0FAFC743F6AD1
:1040DB0070030241D7EEFAEFFB790212205CEE245B
:1040EB000AFEEF3400FFA380E1E0A2E75003024198
:1040FB00D7901040E0A2E450030241D790103CE06F
:10410B00D2E7F0901047E4F0A3F075088F75090122
:10411B00780812034C7CDE7A007B007914121F7036
:10412B0074021202751223937E487F1990103AE0A5
:10413B00F8A3E0F9E875F006A4F8AAF075F006E923
:10414B00A42AF9E82400FAE93419FBEAF8EBF97C24
:10415B00DA7D1975080588828983E493F5098E82C7
:10416B008F83F0EC240BF582ED3400F583E509F039
:10417B008C828D83A3AC82AD8388828983A3A88232
:10418B00A9838E828F83A3AE82AF831508E5087057
:10419B00C58A828B83A3A3A3A3A3E49390194DF0A9
:1041AB00901047E4F0A3F07582487583197E64FF85
:1041BB008012EEFAEFFB790212205CEE240AFEEF7E
:1041CB003400FFA3E0FAFC743F6A70E6901047E4FA
:1041DB00F0A374F8F090103CE0A2E75038C2B07432
:1041EB0080901A40F090104574E0F0A37407F075BE
:1041FB0082CB7583197E647F00E0FAFC743F6A60A2
:10420B0069EEFAEFFB79E112205CEE240AFEEF3443
:10421B0000FFA380E490103DE0FAE0FBEAA2E0503F
:10422B0009EBA2E150047440800CE0A2E04005E0F1
:10423B00A2E150067480901A40F0D2B090104574F1
:10424B00FFF0A3F07582CB7583197E647F0080121B
:10425B00EEFAEFFB79E112205CEE240AFEEF34005C
:10426B00FFA3E0FAFC743F6A70E6901047E4F0A3FA
:10427B0002443212247090103EE0C2E0F07E947F34
:10428B00007508087C0D7D00EEFAEFFB79E1122238
:10429B00FD7C0D7D0074012EFAE43FFB79E11222C7
:1042AB00FDEE240AFEEF3400FF1508E50870D590EB
:1042BB001047E4F0A374F8F090104574FFF0A3F0EE
:1042CB007E007F007508968E098015AA08AB0979C8
:1042DB00E112205CE508240AF508E5093400F5092C
:1042EB00EE2416F582EF341AF583E0FAEE24010E74
:1042FB00EF3400FFEAFC743F6A70D0901047E4F093
:10430B00A3F0FA901047F0A374F8F0901040E0A2DD
:10431B00E440030A8006E0A2E540011AEA25EAF52B
:10432B00EA02427512247090103EE0C2E0F07EE487
:10433B007F007508087C0D7D00EEFAEFFB79E1122A
:10434B0022FD7C0D7D0074012EFAE43FFB79E11216
:10435B0022FDEE240AFEEF3400FF1508E50870D5A8
:10436B00901047E4F0A374F8F090104574FFF0A39D
:10437B00F07E007F007508E68E098015AA08AB0950
:10438B0079E112205CE508240AF508E5093400F50B
:10439B0009EE2420F582EF341AF583E0FAEE2401BE
:1043AB000EEF3400FFEAFC743F6A70D0901047E4C4
:1043BB00F0A3F0FA901047F0A374F8F0901040E0DF
:1043CB00A2E440030A8006E0A2E540011AEA25FCBC
:1043DB00F5FC024275AA08AB0979E112205CE508ED
:1043EB00240AF508E5093400F509EE242AF582EFD5
:1043FB00341AF583E0FAEE24010EEF3400FFEAFCE9
:10440B00743F6A70D0901047E4F0A3F0901040E036
:10441B00A2E4400890103DE0D2E2800BE0A2E54020
:10442B000790103DE0C2E2F0901047E4F0A3F0904B
:10443B001049E50AF0A3E50BF07F0502031474F7AE
:10444B001202B490103CE0A2E750030245349010E6
:10445B0040E0A2E05005E0A2E14025901047E4F0D7
:10446B00A3F075088F750901780812034C7CDE7A6E
:10447B00007B007914121F707402120275122393C1
:10448B0090103DE0FAE0FBEAA2E05025EBA2E150F0
:10449B0020901040E0A2E0400790103DE0C2E0F019
:1044AB00901040E0A2E1405C90103DE0C2E1F08052
:1044BB0053E0A2E0501F901040E0A2E040079010A4
:1044CB003DE0C2E0F0901040E0A2E1403790103D9B
:1044DB00E0D2E180D9E0A2E1901040E05015A2E0DB
:1044EB00400790103DE0D2E0F0901040E0A2E14098
:1044FB001380B5A2E0400890103DE0D2E080AFE021
:10450B00A2E150C990103DE0FAE0FBEAA2E05009AD
:10451B00EBA2E150047440800CE0A2E04005E0A265
:10452B00E150067480901A40F07F0202031474F776
:10453B001202B490104574FFF0A3F0901040E0A26B
:10454B00E450030245DA901041E0A2E090103A509B
:10455B0025E02401F0A3E03400F090103AC3E0947E
:10456B001CA3E09400A2D265D033403C90103A7467
:10457B001BF0A3E48031C3E09418A3E09400A2D213
:10458B0065D03390103AE040102401F0A3E03400E2
:10459B00F0901041E0D2E0800E2401F0A3E0340053
:1045AB00F0901041E0C2E0F0901041E0C2E1F0E089
:1045BB00A2E150547418901038F07440901039F0F8
:1045CB00740290102FF0901041E0D2E20246B5E059
:1045DB00A2E5402B90103AE024FFF0F8A3E034FF63
:1045EB00F0F9C3E89401E99400A2D265D03350B836
:1045FB0090103AE4F0A3F0901041E0D2E180AF903C
:10460B001047E4F0A30247A2E0A2E0504C90103A0E
:10461B00E0F508A3E0F5097808120393180003608E
:10462B0046344647464B4654467418901038F0E4CF
:10463B00901039F0901041E0C2E080187418800B94
:10464B007419901038F0E480087419901038F074D5
:10465B0080901039F07402804EE0A2E2500474187E
:10466B0080E090103AE0F8A3E0F9E8C333F8E933BF
:10467B00F9E82420F582E93418F583E493C0E0745B
:10468B000193F583D082AA82AB838A088B097402CB
:10469B00780812023CE508901038F0EAC433335422
:1046AB00C0901039F0740190102FF07508007E48FF
:1046BB007F1990103AE0F8A3E0F9E875F006A4F83A
:1046CB00AAF075F006E9A42AF9E82400FAE93419EE
:1046DB00FBE82458F8E93418F97CDA7D1990103C82
:1046EB00E0A2E750068A828B83800488828983E468
:1046FB00938E828F83F0E508C394055010E0C0E0E1
:10470B00EC240BF582ED3400F583D0E0F005088C3A
:10471B00828D83A3AC82AD8388828983A3A882A96F
:10472B00838A828B83A3AA82AB838E828F83A3AE71
:10473B0082AF83E508C3940640A3901047E4F0A32F
:10474B0074F8F07582487583197E647F008012EED1
:10475B00FAEFFB790212205CEE240AFEEF3400FF25
:10476B00A3E0FAFC743F6A70E6901047E4F0A3F004
:10477B00901038E0901030F0901039E0901031F03C
:10478B0090103CE0C2E3F0E0D2E2F090103FE0D2B8
:10479B00E1F074599019D8F002453474F81202B450
:1047AB00901040E0A2E04047901000E060109010A5
:1047BB004574E6F0A374FFF0E4901000800A7402D5
:1047CB00F090104574FFF0A3F07582D07583197EBD
:1047DB001E7F00E0FAFC743F6A6063EEFAEFFB7930
:1047EB00E112205CEE240AFEEF3400FFA380E4E02C
:1047FB00A2E1404A901000E06401601190104574F2
:10480B00BFF0A3741DF07401901000800A7402F0C5
:10481B0090104574FFF0A3F07582D07583197E1E3E
:10482B007F008012EEFAEFFB79E112205CEE240A96
:10483B00FEEF3400FFA3E0FAFC743F6A70E69010C1
:10484B0047E4F0A3F090104574FFF0A3F00222F8B8
:10485B0074F41202B4E96003024978901040E0A2AC
:10486B00E4400F901A41E004F0C39408401A740717
:10487B008015E0A2E55003024AA1901A41E0FA74B8
:10488B00FF2AF0EA7002E4F0750848750919E0FE9A
:10489B0075F005A424F8FAE5F03417FBEAF8EBF908
:1048AB007CDA7D19750A0488828983E493F50B857C
:1048BB000882850983F0EC2415F582ED3400F5832D
:1048CB00E50BF08C828D83A3AC82AD8388828983C8
:1048DB00A3A882A983850882850983A3858208857D
:1048EB008309150AE50A70BF8A828B83A3A3A3A34E
:1048FB00E49390194CF07582487583197508C87547
:10490B0009008016AA08AB09790212205CE508247D
:10491B000AF508E5093400F509A3E0FAFC743F6ACF
:10492B0070E2901A41E0C39405901033E04004D23A
:10493B00E08002C2E0F090103FE054EDF0901033B5
:10494B00E090102FF0795D12287490103FE054ED39
:10495B00F0EEC333FEE433FFEE24E8F582EF3417B9
:10496B00F583E49390102FF07948024A8F74016914
:10497B006003024A92901040E0A2E4400F901A426A
:10498B00E004F0C39408401A74078015E0A2E550C8
:10499B0003024AA1901A42E0FA74FF2AF0EA70026D
:1049AB00E4F0750848750919E0FE75F005A424F8C4
:1049BB00FAE5F03417FBEAF8EBF97CDA7D19750AA6
:1049CB000488828983E493F50B850882850983F03B
:1049DB00EC241FF582ED3400F583E50BF08C828D12
:1049EB0083A3AC82AD8388828983A3A882A98385A4
:1049FB000882850983A3858208858309150AE50A40
:104A0B0070BF8A828B83A3A3A3A3E49390194CF06A
:104A1B0075824875831975082C7509018016AA08CB
:104A2B00AB09790212205CE508240AF508E5093484
:104A3B0000F509A3E0FAFC743F6A70E2901A42E0B9
:104A4B00C39405901033E04004D2E08002C2E0F042
:104A5B0090103FE054EDF0901033E090102FF07970
:104A6B005D12287490103FE054EDF0EEC333FEE47A
:104A7B0033FFEE24E8F582EF3417F583E4939010BF
:104A8B002FF07949122874901047E4F0A3F090109E
:094A9B004574FFF0A3F00244444D
:040000050000009166
:00000001FF
